:020000040000FA
:0600000007309F008C2A6E
:08000800A500030EA6008B1AEF
:100010002B280B1A1B28260E8300A50E250E09007F
:1000200081018316640008308100831285149030AA
:100030008B00A40108008B100C30A000A00B1E2820
:1000400006180B28AD30810020308B000230A40050
:100050000830A0000B280B1124193E28A008031912
:100060003728060CA10CA003AD3081000B28061C1C
:1000700058280130A4002108A2005828A4195828A3
:10008000A00803195028A30C031C4928000085145C
:100090004C28851000000000A003B53081000B281B
:1000A0000000000000008514A415A83081000B2872
:1000B00010308B000130A4050B2885100630A400F9
:1000C0000000B5308100A0308B000830A00008008F
:1000D00018300605B50006300605B3003402031DCE
:1000E0007A2035083602031DA0203308B4003508F5
:1000F000B600080034083306063C0319C628330D41
:10010000B40634199228AB08031D9028AC08031DCF
:100110008F282708AB002808AC00AB080319AC03F4
:10012000AB030800AB0A0319AC0A27082B02031D16
:10013000080028082C02031D0800AB01AC010800D0
:1001400036083506183C0319C628350DB606361A8A
:10015000B828AD08031DB628AE08031DB528290828
:10016000AD002A08AE00AD080319AE03AD030800C8
:10017000AD0A0319AE0A29082D02031D08002A083A
:100180002E02031D0800AD01AE010800B70A0800E9
:100190004D22241CC828241008005D204D22A418DC
:1001A000CE2808002908AD002A08AE000310AE0CC6
:1001B000AD0C2708AB002808AC000310AC0CAB0C4E
:1001C0000800C8202208A700C8202208A800C820CC
:1001D0002208A900C8202208AA00D2207230A30059
:1001E000CD200321A02A15213B08A9003A08AA0026
:1001F00015213B08A7003A08A800D2203E08A3001A
:10020000CD200321A02A273084000030712229301C
:1002100084000230712208002730840000306222FE
:100220002930840002306222080040308400BD0181
:10023000BB01BA01BD08031D3729C8202208203C94
:1002400003191A292208093C03191A2922080D3C0E
:1002500003191A2922082B3C03191A2922082D3CBC
:1002600003191A2922088000BD0A840A1D29840363
:100270000030B8000130B9006221BD0B40290800F0
:1002800084030030B8000A30B9006221BD0B49294F
:10029000080084030030B8006430B9006221BD0B4F
:1002A0005229080084030330B800E830B900622105
:1002B000BD0B5B29080084032730B8001030B9005B
:1002C000622108002F300002BC00BC0B6829080026
:1002D0003908BB070318BA0A3808BA07652937086E
:1002E000A300CD20B701A02A3708303EA300CD20BF
:1002F0003030A300CD203130A300CD20B701A02A9B
:100300003708B900B8012622B701A02A2B08AF0090
:100310002C08B0002D08B1002E08B2002F08A30051
:10032000CD203008A300CD203108A300CD20320815
:10033000A300CD20A02A2B08AF002C08B0002D0868
:10034000B1002E08B2003E08523C031DAF29AA1F7F
:10035000AF293108B9003208B800ED21BF292908BA
:10036000B9002A08B8000310B80CB90C39083102DA
:10037000031CB203B90038083202B800E221093088
:10038000A300CD203E08523C031DCE29A81FCE2934
:100390002F08B9003008B800ED21DE292708B90080
:1003A0002808B8000310B80CB90C39082F02031C38
:1003B000B003B90038083002B800E2210D30A300C4
:1003C000CD20A02AB81FED29B809B909B90A031927
:1003D000B80A2D30A300CD20F0292B30A300CD206A
:1003E000162208002708A300CD202808A300CD204E
:1003F0002908A300CD202A08A300CD20A02A2B3055
:10040000A300CD202A08B8002908B9001622093017
:10041000A300CD202B30A300CD202808B80027084A
:10042000B90016220D30A300CD20A02A2730BA0033
:100430001030BB003B223C08A300CD200330BA00A3
:10044000E830BB003B223C08A300CD200030BA00BE
:100450006430BB003B223C08A300CD200030BA0032
:100460000A30BB003B223C08A300CD203908303EB7
:10047000A300CD2008002F30BC00BC0A3B08B90205
:100480003A08031C013EB80203183D2A3B08B9078D
:100490003A080318013EB8070800682008005630E3
:1004A000A300CD203230A300CD202E30A300CD20DC
:1004B0003030A300CD203130A300CD200D30A3007B
:1004C000CD20080083169B0083120230C6008316DD
:1004D0001C141A089B0A8000840A8312C60B672A20
:1004E000080083169B0083120230C6008B1383160C
:1004F00000089A009C011C1555309D00AA309D00F3
:100500009C149C18812A9C139B0A83128C13840AC6
:10051000C60B772A8B17080083161F308600003021
:10052000850083128501102006300605B4001830BE
:100530000605B6000C21B701D2204E30BF004F2275
:10054000A201C8202208793C0319862922087A3C96
:100550000319E1282208703C03196F292208683C1E
:100560000319F22922085A3C031DB92A2A30BE0079
:10057000F3282208523C031DC02A5230BE00F32843
:100580002208723C031DC72A5230BE00F3282208FD
:10059000483C0319FF292208513C03199B292208D2
:1005A000503C031974292208413C031DDA2A5930B2
:1005B000BF00A02A2208613C031DE22A3F08A300D5
:0E05C000CD20A02A2208713C03198029A02A10
:0205CE000034F7
:0205D0000034F5
:02400E00013F70
:00000001FF
